:100000000C948F060C94AC060C94AC060C94AC06C5
:100010000C94AC060C94AC060C94AC060C94AC0698
:100020000C94AC060C94AC060C94272C0C94F92C74
:100030000C948E260C94AC060C94AC060C94AC0676
:100040000C94AC060C94AC060C94AC060C94AC0668
:100050000C94AC060C9416270C94AC060C94AC06CD
:100060000C94AC060C94AC060C94AC060C94AC0648
:100070000C94AC060C94AC060C94AC060C94AC0638
:100080000C94AC060C94AC060C94AC060C94AC0628
:100090000C94AC060C94AC060C94AC060C94AC0618
:1000A0000C94AC060C94AC060C94AC06780A780A56
:1000B000A40AA40A0C0B370C370C370C2A0BC30B01
:1000C000D40BD40B662D8D2D852E8D2D852ED92DFF
:1000D000FC2D852E532E622E01515200A800500097
:1000E00051004F0001004A00005CAC004D00AB0025
:1000F00044454255473A2064697361626C65642ED9
:100100000A0044454255473A20656E61626C656459
:100110002E0A000A0025303258006C65645F746155
:10012000736B3A20004F6E6573686F743A20616399
:10013000746976653A2025640A000A002530386221
:10014000003A200025303258000A722F63203031E7
:100150003233343536370A007267626C6967687407
:100160002074696D65722064697361626C652E0A22
:10017000007267626C696768742074696D657220CB
:10018000656E61626C65642E0A007267626C6967F5
:1001900068742073657420687376205B4E4F454504
:1001A00050524F4D5D3A2025752C25752C25750A2A
:1001B000007267626C696768742073657420687385
:1001C00076205B454550524F4D5D3A2025752C25D4
:1001D000752C25750A007267626C696768742072F5
:1001E00061696E626F7720736574206873763A2058
:1001F00025642C25642C25642C25750A0072676201
:100200006C696768742064697361626C65205B4E19
:100210004F454550524F4D5D3A207267626C696799
:1002200068745F636F6E6669672E656E61626C6588
:10023000203D2025750A007267626C69676874202A
:1002400064697361626C65205B454550524F4D5D3A
:100250003A207267626C696768745F636F6E666983
:10026000672E656E61626C65203D2025750A0072FF
:1002700067626C6967687420656E61626C65205B9B
:100280004E4F454550524F4D5D3A207267626C6942
:100290006768745F636F6E6669672E656E61626C16
:1002A00065203D2025750A007267626C6967687475
:1002B00020656E61626C65205B454550524F4D5D17
:1002C0003A207267626C696768745F636F6E666913
:1002D000672E656E61626C65203D2025750A00728F
:1002E00067626C6967687420746F67676C65205B10
:1002F000454550524F4D5D3A207267626C696768A0
:10030000745F636F6E6669672E656E61626C6520EF
:100310003D2025750A007267626C69676874206DFC
:100320006F6465205B4E4F454550524F4D5D3A20FE
:1003300025750A007267626C69676874206D6F6466
:1003400065205B454550524F4D5D3A2025750A00AA
:100350007267626C696768745F696E69742072673E
:10036000626C696768745F636F6E6669672E6D6F34
:100370006465203D20302E205772697465206465C5
:100380006661756C742076616C75657320746F207E
:10039000454550524F4D2E0A007267626C6967687E
:1003A000745F696E6974206565636F6E6669672046
:1003B0006973206E6F7420656E61626C65642E0ACD
:1003C000007267626C696768745F696E6974207334
:1003D00074617274210A007267626C696768745F85
:1003E000696E69742063616C6C65642E0A007267C3
:1003F000626C696768745F636F6E6669672E73709D
:10040000656564203D2025640A007267626C696737
:1004100068745F636F6E6669672E76616C203D203D
:1004200025640A007267626C696768745F636F6E47
:100430006669672E736174203D2025640A00726727
:10044000626C696768745F636F6E6669672E687552
:1004500065203D2025640A007267686C69676874CE
:100460005F636F6E6669672E6D6F6465203D202542
:10047000640A007267626C696768745F636F6E66B6
:1004800069672E656E61626C65203D2025640A00F7
:100490007267626C696768745F636F6E6669672014
:1004A000454550524F4D3A0A0000047F3F1F6432C9
:1004B00014643214783C1E1E140A052223252628B3
:1004C000292A2C2D2F3032333536383A3B3D3E40E9
:1004D00042434547494A4C4E5051535557595A5C2F
:1004E0005E6062646668696B6D6F71737577797B46
:1004F0007D7F81838587898A8C8E90929496989A45
:100500009C9E9FA1A3A5A7A8AAACAEAFB1B3B4B659
:10051000B8B9BBBCBEBFC1C2C3C5C6C7C9CACBCCB4
:10052000CDCED0D1D2D2D3D4D5D6D7D7D8D9D9DA87
:10053000DADBDBDBDCDCDCDCDCDDDDDDDDDCDCDCFC
:10054000DCDCDBDBDBDADAD9D9D8D7D7D6D5D4D324
:10055000D2D2D1D0CECDCCCBCAC9C7C6C5C3C2C1F9
:10056000BFBEBCBBB9B8B6B4B3B1AFAEACAAA8A756
:10057000A5A3A19F9E9C9A98969492908E8C8A890E
:10058000878583817F7D7B79777573716F6D6B69EB
:1005900068666462605E5C5A5957555351504E4CC0
:1005A0004A4947454342403E3D3B3A38363533326F
:1005B000302F2D2C2A292826252322FFAA7F5540BB
:1005C0000001010101010101010102020202020216
:1005D00002020203030303030303030404040404E9
:1005E00004040505050505060606060607070707B0
:1005F0000708080808090909090A0A0A0B0B0B0C65
:100600000C0C0D0D0D0E0E0E0F0F0F101011111101
:100610001212131314141515161617171818191982
:100620001A1A1B1B1C1D1D1E1E1F202021222223E7
:100630002424252626272829292A2B2C2D2D2E2F28
:1006400030313232333435363738393A3B3C3D3E3F
:100650003F404142434445464748494A4C4D4E4F2E
:1006600050515354555658595A5B5D5E5F616264F0
:10067000656668696B6C6D6F7072737577787A7B7D
:100680007D7E8082838587888A8C8E8F91939596D4
:10069000989A9C9EA0A2A3A5A7A9ABADAFB1B3B5F4
:1006A000B7BABCBEC0C2C4C6C9CBCDCFD1D4D6D8D0
:1006B000DBDDDFE2E4E7E9EBEEF0F3F5F8FAFDFF6E
:1006C0003F00433E20004C25640A000A092D2053B8
:1006D0007461747573202D0A686F73745F6B65792C
:1006E000626F6172645F6C65647328293A202530FB
:1006F00032580A6B6579626F6172645F70726F74F1
:100700006F636F6C3A20253032580A6B6579626FDF
:100710006172645F69646C653A20253032580A74EE
:10072000696D65725F72656164333228293A2025EC
:1007300030386C580A000A092D2056657273696FAB
:100740006E202D0A5649443A2030784645454428C3
:1007500047686F7374536576656E29205049443A33
:10076000203078444144332842656E746F204D61D7
:1007700063726F706164205265762E203129205695
:1007800045523A203078303130300A4255494C4495
:100790003A20202846656220323720323032322912
:1007A0000A4F5054494F4E533A204C55464120452C
:1007B000585452414B455920434F4E534F4C4520BE
:1007C000434F4D4D414E4420343039360A47434360
:1007D0003A20352E342E30204156522D4C4942437A
:1007E0003A20322E302E30204156525F415243483B
:1007F0003A20617672350A000A092D20436F6E7324
:100800006F6C65202D0A4553432F713A0971756944
:10081000740A000A092D204D61676963202D0A447E
:100820003A094465627567204D6573736167652099
:10083000546F67676C650A583A094D61747269783C
:10084000204465627567204D6F646520546F67674B
:100850006C65202D2053686F77206B657970726509
:100860007373657320696E206D6174726978206797
:100870007269640A4B3A094B6579626F6172642050
:10088000446562756720546F67676C65202D20533F
:10089000686F77206B65797072657373207265700D
:1008A0006F72740A4D3A094465627567204D6F7521
:1008B000736520546F67676C650A563A095665720E
:1008C00073696F6E0A533A095374617475730A43FE
:1008D0003A09416374697661746520436F6E736F82
:1008E0006C65204D6F64650A46312D4631303A09FA
:1008F00053776974636820746F204C617965722046
:10090000302D392028463130203D204C30290A3006
:100910002D393A0953776974636820746F204C61EC
:1009200079657220302D390A47524156453A0953AC
:10093000776974636820746F204C61796572203028
:100940002028616C7465726E617465290A423A09E7
:100950004A756D7020746F20426F6F746C6F6164A4
:1009600065720A4553433A094A756D7020746F20C9
:10097000426F6F746C6F616465722028616C74657E
:10098000726E617465290A453A095072696E742065
:10099000454550524F4D2053657474696E67730A14
:1009A0004253504143453A09436C656172204545C5
:1009B00050524F4D0A006B65796D61705F636F6EC9
:1009C0006669672E7261773A20253032580A2E7395
:1009D0007761705F636F6E74726F6C5F6361707369
:1009E0006C6F636B3A2025750A2E636170736C6FB0
:1009F000636B5F746F5F636F6E74726F6C3A202508
:100A0000750A2E737761705F6C63746C5F6C6775C9
:100A1000693A2025750A2E737761705F7263746C72
:100A20005F726775693A2025750A2E737761705F6A
:100A30006C616C745F6C6775693A2025750A2E735A
:100A40007761705F72616C745F726775693A2025B7
:100A5000750A2E6E6F5F6775693A2025750A2E73C9
:100A60007761705F67726176655F6573633A2025B1
:100A7000750A2E737761705F6261636B736C61736B
:100A8000685F6261636B73706163653A2025750A04
:100A90002E6E6B726F3A2025750A00646562756769
:100AA0005F636F6E6669672E7261773A2025303218
:100AB000580A2E656E61626C653A2025750A2E6DA6
:100AC00061747269783A2025750A2E6B6579626FB8
:100AD0006172643A2025750A2E6D6F7573653A2030
:100AE00025750A006565636F6E6669673A0A646515
:100AF0006661756C745F6C617965723A2025750A60
:100B0000003F000A6D6F7573653A206F66660A00D4
:100B10000A6D6F7573653A206F6E0A000A6B65790E
:100B2000626F6172643A206F66660A000A6B6579CB
:100B3000626F6172643A206F6E0A000A6D617472AE
:100B400069783A206F66660A000A6D617472697886
:100B50003A206F6E0A000A64656275673A206F6614
:100B6000660A000A64656275673A206F6E0A000AB9
:100B70000A4A756D70696E6720746F20626F6F74BA
:100B80006C6F616465722E2E2E2000433E20004360
:100B90006C656172696E6720454550524F4D0A0081
:100BA0000A002530325820006B6579626F617264EB
:100BB0005F7265706F72743A20005B735D005B5703
:100BC0005D005B535D005B525D005B445D005B4319
:100BD0005D002C03420065006E0074006F00200071
:100BE0004D006100630072006F00700061006400DE
:100BF00020005200650076002E0020003100000029
:100C00001603470068006F0073007400530065000E
:100C1000760065006E0000000403090409025B0011
:100C2000030100A0FA0904000001030101000921E9
:100C30001101000122400007058103080001090499
:100C4000010001030000000921110100012232000E
:100C500007058203200001090402000203000000CE
:100C60000921110100012222000705830320000150
:100C7000070503032000011201000200000008ED37
:100C8000FED3DA0001010200010631FF0974A1015F
:100C90000975150026FF0095207508810209761553
:100CA0000026FF00952075089102C005010980A16A
:100CB00001850319012AB700150126B700950175B2
:100CC000108100C0050C0901A101850419012AA0A9
:100CD00002150126A002950175108100C0050109C9
:100CE00006A101050719E029E715002501950875FA
:100CF0000181029501750881010507190029FF1579
:100D00000026FF00950675088100050819012905D0
:100D1000950575019102950175039101C00011249B
:100D20001FBECFEFDAE0DEBFCDBF11E0A0E0B1E043
:100D3000E2E5FFE502C005900D92A03DB107D9F7AD
:100D400022E0A0EDB1E001C01D92A539B207E1F7A4
:100D50000E94F2170C94A72F0C940000FF93EF93BE
:100D6000E091D001F091D101309709F00995EF9110
:100D7000FF910895FC018591803011F0EFDFFBCFEA
:100D80000895FF27E0E230E247FF0CC0419597FF4E
:100D900009C0EDE26095709580959095611D711D7B
:100DA000811D911D27FF02C0219530E350E2AA2743
:100DB000660F771F881F991FAA1FA41710F0A41B86
:100DC00063955A95A9F7AA3008F0A95FA05DAF9383
:100DD000F395611571058105910541F7ED3211F427
:100DE000EF93F395F21718F43F93F395FBCF8F91A0
:100DF000B5DFFA95E1F70895E991F9918591803091
:100E000021F0853219F0AADFF9CF089520E0E894A7
:100E100055915532C1F3503311F4689455915A33BA
:100E200048F4505390F3220F022E220F220F200D70
:100E3000250FF4CF0EF4219589919991533619F32A
:100E4000533729F1533559F1BC0188279927E89484
:100E50005C3621F48991999168945591543639F40E
:100E600046EF7EF077FF0DC08FEF9FEF0AC055373A
:100E70004AE039F0583540E121F0523642E009F0BD
:100E80000895FF93EF937DDFEF91FF91B7CFFF932D
:100E9000EF93FC0181918030B9F360DFFBCFFF93CA
:100EA000EF9368DFF1CFDF93CF93CDB7DEB7259611
:100EB000A3DFCF91DF9108950E942A1E4FEF6FEFBD
:100EC00080E00E94881B8BE00E94271E0C94441334
:100ED000811107C0662311F089EA01C08AEA0E94E5
:100EE000260A81E0089581E0089581E008950C9438
:100EF000750708950C9479071F93CF93DF9300D063
:100F000000D01F92CDB7DEB749835A836B833091EF
:100F1000D30189819A81311114C0662359F02223AB
:100F200049F00E94700E182F682F89819A810E94C3
:100F3000190E03C00E94440E182F69817A81812FF7
:100F400004C00E94700E69817A810F900F900F90FB
:100F50000F900F90DF91CF911F910C949E15FC0183
:100F6000262F408151816281738184810C947C079A
:100F700081E00895CF93DF93EC0160E00E94AF071A
:100F8000BE01DF91CF910C947A070C9408170C9452
:100F9000041708950E94C30C0E94C9072FEF84E331
:100FA0009CE0215080409040E1F700C000000C948C
:100FB0003C270F931F93CF93DF938C0161E00E9436
:100FC000AF07EC01B8010E947707882309F462C0DB
:100FD000B801CE010E942825882309F45BC0B8011E
:100FE000CE010E94F620882309F454C0B801CE0136
:100FF0000E948424882309F44DC0B801CE010E94C8
:10100000FC1F882309F446C0F80182818823D9F1A6
:10101000CF3D8CE5D80779F140F4C115FCE5DF0739
:1010200091F0C130DC4591F02EC0CC35EDE5DE0706
:1010300041F1CD35FDE5DF0709F1CB35DD4519F58A
:101040000E94071320C00E94CA0724C080913B025F
:10105000C82FC095C170C0FB80F980933B02CC23A0
:1010600029F082E091E00E94BA0614C080EF90E07F
:101070000E94BA0610C00E94A8130CC00E94FE1263
:1010800002C00E940A13C801DF91CF911F910F91F6
:101090000C947307C0E08C2FDF91CF911F910F91BB
:1010A00008950E946F260E9480080C943D1F0E94A4
:1010B00083080E94C81E0C9475268295982F9373FE
:1010C00044E0949F900111248C7C86958695282B72
:1010D000822F8575880F2A7A2695822B0895089588
:1010E0000C946F0881E008950C9472080895CF93D2
:1010F000C82F0E9470088C2F0E947408CF91089509
:1011000080E00C9477080E9484250C947708CF9394
:101110000E948425C82F8091D201C81741F1C09345
:10112000D20180913B0282FF1EC080FF04C08AE191
:1011300091E00E94BA0680913B0280FF0CC01F9292
:10114000CF9385E191E09F938F930E9453070F9077
:101150000F900F900F9080913B0280FF04C083E1BD
:1011600091E00E94BA068C2FCF910C947708CF9112
:101170000895CF93DF93CDB7DEB72B970FB6F894D2
:10118000DEBF0FBECDBF4F83588769877A878B87B5
:1011900061110E9436129E012F5F3F4F86E0F901D8
:1011A00011928A95E9F785E0FE013796D901019001
:1011B0000D928A95E1F789819A814C815D81452B59
:1011C00031F09F3F31F491E08F3F19F403C091E07B
:1011D00001C090E090FF09C049815A816B817C81F8
:1011E0008D819E810E94571105C0C9010E94B807D8
:1011F0008111F2CF2B960FB6F894DEBF0FBECDBF94
:10120000DF91CF910895FC01808191810E94B20EFF
:101210000895CF93882309F4A1C0C82F8238C1F460
:101220000E94842581FD9AC069E38091020190911A
:1012300003010E9447260E9458122FEF81EE94E08E
:10124000215080409040E1F700C0000069E319C0E0
:10125000833801F50E94842580FD80C063E580917C
:101260000201909103010E9447260E9458122FEF1D
:1012700081EE94E0215080409040E1F700C00000F2
:1012800063E580910201909103010E944926CF916C
:101290000C9458128438C1F40E94842582FD5EC0EB
:1012A00067E480910201909103010E9447260E9409
:1012B00058122FEF81EE94E0215080409040E1F7EA
:1012C00000C0000067E4DDCF8CEF8C0F813AF8F4AA
:1012D0008C2F0E94D523811141C06C2F8091020177
:1012E000909103010E941126882349F06C2F809170
:1012F0000201909103010E9449260E9458126C2F0E
:1013000080910201909103010E944726C0CF80E2A4
:101310008C0F883048F4C77081E001C0880FCA95EF
:10132000EAF70E941912B3CFEBE5EC0FE33040F47B
:10133000F0E0EE5AFE4F808190E0CF910C94D925D9
:10134000C85AC73158F4EC2FF0E0EE0FFF1FEC5DE8
:10135000FE4F80819181CF910C94EF25CF9108951C
:10136000882309F45BC0682F823879F40E948425B1
:1013700081FF54C069E380910201909103010E94B2
:1013800047260E94581269E310C08338B1F40E94C6
:10139000842580FF43C063E58091020190910301A1
:1013A0000E9447260E94581263E5809102019091A5
:1013B00003010E9449260C945812843879F40E9443
:1013C000842582FF2BC067E4809102019091030184
:1013D0000E9447260E94581267E4E7CF8CEF860FE1
:1013E000813A18F380E2860F883048F4677081E014
:1013F00001C0880F6A95EAF70E941F12DCCF8BE5C7
:10140000860F833020F480E090E00C94D925685A50
:10141000673120F480E090E00C94EF2508951F934D
:10142000CF93DF93182FEB010E940909209741F019
:101430008FE99FE00197F1F700C000002197F6CFF8
:10144000812FDF91CF911F910C94B009893319F04E
:1014500060E070E002C060E570E00C940F0A882341
:1014600021F00E9419120C9458120895882321F03B
:101470000E941F120C9458120895CF92DF92EF929F
:10148000FF920F931F93CF93DF937C01D62FC72F2B
:10149000FC011281058102950F700E940F128823B2
:1014A000B9F01123A9F08C2F807F803421F080E2E5
:1014B0008D0F883068F080916E0282FD09C082E055
:1014C0000E94B8120E940F1291E0D82ED92601C0B6
:1014D000D12CCC2EC2948FE0C8228C2D90E08C3081
:1014E000910508F0C4C1FC01EA5AFF4F0C940E2F7D
:1014F0008C2F807FCF70882311F0C295C07F11237D
:1015000099F0CC2309F49FC180E28D0F883010F050
:10151000D11104C08C2F0E94191203C08C2F0E947D
:1015200029120E9458128FC18D2F0E94B009CC231E
:1015300009F49DC180E28D0F883038F1DD2329F157
:101540008C2F0E942F1224C08C2F807FCF7080326E
:1015500011F0C295C07FDD2319F0D130A1F13DC05B
:1015600080916E0282FF17C0112349F0CC2329F02D
:101570008C2F0E9419120E94581280E065C180E0F1
:101580000E94B009CC2309F472C18C2F0E941F1253
:101590000E9458126CC1112371F0002341F00130F8
:1015A00031F40E9439128C2B0E94411260C10E94BA
:1015B00039128C2B1DC0002319F0013009F457C1DA
:1015C0000E944E1225C0112321F0063008F04FC1B1
:1015D0000EC0053008F04BC11BC0112361F0002381
:1015E00031F0F701858180FF2EC18F7085838C2FAC
:1015F0000E942F0A3CC1002359F0D93309F034C1AD
:10160000FFEF07EE13E0F15000401040E1F72AC170
:101610008C2F0E94360A2BC18C2F8695869583705D
:1016200019F0813061F023C1112321F08D2F9C2FFF
:10163000937002C080E090E00E94D92520C1112360
:1016400021F08D2F9C2F937002C080E090E00E94CB
:10165000EF2515C18C2F837009F047C011110BC104
:101660002D2F229526952770220F220F6D2F6F7038
:10167000862F90E0A0E0B0E0022E04C0880F991FF2
:10168000AA1FBB1F0A94D2F7D4FF10C04FE050E04E
:1016900060E070E004C0440F551F661F771F2A9555
:1016A000D2F7409550956095709503C040E050E0AA
:1016B000BA01C695C695C3708A019B01082B192BE8
:1016C0002A2B3B2BC901B801C23049F058F4C13074
:1016D00019F00E942F0DCFC00E941D0DCCC00E949A
:1016E000410DC9C00E941B0DC6C0112319F08C2FDB
:1016F000817001C08695882309F4BDC02D2F2295E5
:1017000026952770220F220F6D2F6F70862F90E085
:10171000A0E0B0E0022E04C0880F991FAA1FBB1FD3
:101720000A94D2F7D4FF10C04FE050E060E070E0C0
:1017300004C0440F551F661F771F2A95D2F74095A6
:1017400050956095709503C040E050E0BA01C69591
:10175000C695C3708A019B01082B192B2A2B3B2BA2
:10176000C901B801C23049F058F4C13019F00E94E3
:10177000F40D81C00E94E20D7EC00E94060E7BC067
:101780000E94550D78C0CF70112339F08C2F0E9424
:101790007B0D8D2F0E942F0A6EC08D2F0E94360A5E
:1017A0008C2F0E949C0D67C0D23F21F128F4D03FBE
:1017B00041F0D13FC1F043C0D33F19F1D43F79F09C
:1017C0003EC0112341F0053008F051C08C2F8F71BD
:1017D0000E94C10D4CC0063008F049C0F7CF80917F
:1017E0006E0282FF18C0112339F08C2F8F710E9476
:1017F0007B0D3DC01123C9F38C2F8F710E949C0D6E
:1018000036C0112329F08C2F8F710E94660D2FC0D6
:101810000E94610D2CC0112349F0CF718C2F0E94C2
:101820007B0D63E08C2F0E949D1221C081E00E94FD
:10183000B8120230E0F082E00E94B81218C0112302
:1018400031F0002391F28D2F0E94090910C000236E
:1018500099F2D93349F41FEF27EE33E011502040BD
:101860003040E1F700C000008D2F0E94B00988EFE2
:101870008C0D843020F40E9484250E947708DD209E
:10188000C9F00E940B1280FD15C0F70112820E9460
:1018900005120E947B0DC7010E947B0C0E9405125D
:1018A000DF91CF911F910F91FF90EF90DF90CF903C
:1018B0000C949C0DDF91CF911F910F91FF90EF90B1
:1018C000DF90CF9008950F931F93CF93DF93EC0198
:1018D000688179818A810E94BD0E8C010E94180E58
:1018E0000E94090DB801CE010E943D0ADF91CF91FF
:1018F0001F910F910895CF93DF93EC019881898117
:101900002B813C81232B31F08F3F31F481E09F3FCD
:1019100019F403C081E001C080E080FD1DC0CE014C
:101920000E94D907811110C00E940F128823A1F0D4
:101930008A81882389F080916E0282FD0DC082E049
:10194000DF91CF910C94B812CE010E94630CCE01AE
:10195000DF91CF910C94BA07DF91CF91089580E089
:1019600090E00E94D92580E090E00E94EF250E943F
:1019700036120C94581280910201909103010E943A
:101980004B260C94AF0C0E9426120C94BB0C929523
:101990009F70963079F010F4925001C09A509230B6
:1019A00068F4803F69F018F4883E40F409C0843F31
:1019B00029F406C0883E20F0813F11F080E00895B0
:1019C00081E00895FC01808191810E94B20E0E9405
:1019D000C70C0895CF93DF9300D000D01F92CDB7EE
:1019E000DEB70F900F900F900F900F90DF91CF9177
:1019F0000895CF93DF9300D000D000D0CDB7DEB7ED
:101A000026960FB6F894DEBF0FBECDBFDF91CF9103
:101A10000895089508950C940A0D0C940B0D0E94DE
:101A20000D0D6093DD017093DE018093DF019093D3
:101A3000E0010C94AF0C0C940F0D0F931F930091C9
:101A4000DD011091DE012091DF013091E001602B7A
:101A5000712B822B932B1F910F910C940F0D0F93D1
:101A60001F930091DD011091DE012091DF01309183
:101A7000E00160237123822393231F910F910C9423
:101A80000F0D0F931F930091DD011091DE01209146
:101A9000DF013091E00160277127822793271F9192
:101AA0000F910C940F0D0C940A0D0E94530D60932E
:101AB000D9017093DA018093DB019093DC010C94DF
:101AC000AF0C60E070E0CB010C94550D0F931F93A9
:101AD00041E050E060E070E08A019B0104C0000F2B
:101AE000111F221F331F8A95D2F7C901B8011F9118
:101AF0000F910C94550D0F931F9341E050E060E05F
:101B000070E004C0440F551F661F771F8A95D2F7F7
:101B10008091D9019091DA01A091DB01B091DC01B3
:101B20008A019B01082B192B2A2B3B2BC901B801D9
:101B30001F910F910C94550D0F931F9341E050E0AE
:101B400060E070E004C0440F551F661F771F8A9540
:101B5000D2F740955095609570958091D9019091FC
:101B6000DA01A091DB01B091DC018A019B0108231D
:101B700019232A233B23C901B8011F910F910C940B
:101B8000550D0F931F9341E050E060E070E004C0FA
:101B9000440F551F661F771F8A95D2F78091D90190
:101BA0009091DA01A091DB01B091DC018A019B01E7
:101BB000082719272A273B27C901B8011F910F9130
:101BC0000C94550D0F931F930091D9011091DA01D8
:101BD0002091DB013091DC01602B712B822B932B48
:101BE0001F910F910C94550D0F931F930091D901E4
:101BF0001091DA012091DB013091DC016023712327
:101C0000822393231F910F910C94550D0F931F93D3
:101C10000091D9011091DA012091DB013091DC01B2
:101C200060277127822793271F910F910C94550DE0
:101C30000895292F220F920F890FE82FE695E69538
:101C4000E695877051E001C0550F8A95EAF785E067
:101C5000E89FF0011124EC52FE4F20E030E070E0EC
:101C60004081CB01022E02C0969587950A94E2F737
:101C70008170819584278523842781932F5F3F4F2F
:101C80002530310569F70895292F220F920F890F0A
:101C9000682F669566956695982F977085E0689F82
:101CA000B001112440E050E080E0FB01E40FF51F9B
:101CB000EC52FE4F208130E0092E02C03695279568
:101CC0000A94E2F721703327042E01C0220F0A94F0
:101CD000EAF7822B4F5F5F4F4530510531F708958A
:101CE000BF92CF92DF92EF92FF920F931F93CF9309
:101CF000DF938C01C090D901D090DA01E090DB0134
:101D0000F090DC018091DD019091DE01A091DF0176
:101D1000B091E001C82AD92AEA2AFB2ACFE1D0E013
:101D2000D701C6010C2E04C0B695A7959795879547
:101D30000A94D2F780FD04C0219790F7B12C07C018
:101D4000BC2EB8018C2F0E94B4150197A9F38B2DDE
:101D5000DF91CF911F910F91FF90EF90DF90CF9087
:101D6000BF900895CF93DF93EC010E94700EBE01E7
:101D70000E94B415DF91CF9108951F93CF93DF9305
:101D8000EB019091D301992321F0CB010E94B20E77
:101D900013C0882349F0CB010E94700E182F682FC2
:101DA000CE010E94190E04C0CB010E94440E182FD0
:101DB000BE01812F0E94B415DF91CF911F9108952C
:101DC0001F93CF93DF93C091E10116E08091E20170
:101DD000C81799F0D0E01C9FF0011D9FF00D112451
:101DE000ED51FE4F408151816281738184819581E3
:101DF0000E94F90C2196C770E9CFDF91CF911F9116
:101E0000089540911302509114026091150270914F
:101E1000160280911702909118020C94F90CEF921F
:101E2000FF920F931F93CF93DF93809118028295B7
:101E30008F7009F065C080911502882309F460C095
:101E40008091E101F090E2011091130200911402DF
:101E5000609116027091170291E01F3F09F090E027
:101E6000C0910001D0910101292F96E0E92E8F1534
:101E700009F446C06115710521F00F3F21F030E0F3
:101E800003C031E001C0322F90E030FD36C0E89E43
:101E9000F001E99EF00D1124DF01AD51BE4F119606
:101EA0003C911197301329C03C91311326C01296F2
:101EB0003C911297311121C013964D915C9114976A
:101EC000461B570B4C175D07C0F4809118028F70AA
:101ED000806180931802E851FE4F80818F7080618D
:101EE000808383E192E00E947B0CDF91CF911F9170
:101EF0000F91FF90EF900C94E00E01968770B7CF92
:101F0000DF91CF911F910F91FF90EF9008959F92D5
:101F1000AF92BF92CF92DF92EF92FF920F931F93F7
:101F2000CF93DF93CDB7DEB761970FB6F894DEBFDE
:101F30000FBECDBF8C0185E0F801DE011D9601903A
:101F40000D928A95E1F7D8011296EC9090911302C8
:101F5000E0911402209116023091170221153105EB
:101F600031F0EF3F31F481E09F3F19F403C081E08D
:101F700001C080E0B82FB1709B2E80FD47C1D80111
:101F80004C9111965C9111971396AD90BC9014975B
:101F900083E1C82E82E0D82EF0901502B501621BB5
:101FA000730B2091000130910101FF2009F4D9C089
:101FB000809118026217730708F095C0282F207FC0
:101FC00009F052C05E1313C0491311C0FE2CE1107A
:101FD0000EC08F708061809318020E94010FC601AD
:101FE0000E947B0C80911802F80185834DC1AB28BB
:101FF00031F05F3F31F481E04F3F19F403C081E0DD
:1020000001C080E080FD03C081E08E2502C080E039
:1020100090E0F82FF170FF2E80FF1CC08091E1014D
:102020002091E20136E0821709F40BC190E0389F5D
:10203000F001399FF00D1124ED51FE4F61815613CF
:1020400006C06081461303C06281E61203C0019698
:102050008770E9CFFE2CEE2009F416C1809118029A
:1020600081608093180254C05E1306C0491304C0F7
:10207000E11002C0F80199C0C8010E94E20C882357
:1020800061F1EE2051F120911802822F82958F701C
:1020900090E0029774F08091130290911402988757
:1020A0008F831986BB86AA862C87CE0107960E944D
:1020B0007B0C86E0F801A3E1B2E001900D928A95D5
:1020C000E1F70E940F0F0E94010F0AC05E1711F185
:1020D000C8010E94E20C81112CC0C8010E947B0C37
:1020E000FF24F394D1C0282F207F81F77A2DB98A5D
:1020F000A88A6E2D89890E94EA0C83E192E00E94F1
:102100007B0C86E0D6011D928A95E9F70E94010FAB
:10211000F12CBAC04913DCCFE110DACFF801858386
:10212000C8010E947B0C86E0D6011D928A95E9F7D2
:10213000ABC0EE2091F220911802822F82958F7011
:1021400090E002970CF4B5CF8091130290911402A5
:102150009A8389831B82BD82AC822E83CE01019635
:10216000A6CF6217730708F044C0FE2CEE2009F4D6
:10217000B4CF5E1330C049132EC02091180220FD49
:1021800021C0822F82958F70482F50E04115510554
:10219000C9F0F80125834F30510541F08F5F982F2A
:1021A0009295907F822F8F70892B8583C8010E9422
:1021B0007B0C86E0F801A3E1B2E001900D928A95D4
:1021C000E1F73CC086E0F801A3E1B2E001900D9296
:1021D0008A95E1F759C0C8010E94E20C811169CFCC
:1021E00080911802816080931802C8010E947B0CC4
:1021F0004BC07A2DB98AA88A6E2D89890E94EA0C73
:1022000086E0D6011D928A95E9F718C0EE2009F400
:1022100064CFC8010E94E20CF82E882309F45DCF38
:1022200086E0F801A3E1B2E001900D928A95E1F712
:1022300083E192E00E9403090E940F0F0E94010FA8
:1022400023C04D875E878D859E850E94B20E292F03
:1022500022952F70223028F49F7039F0811105C02B
:102260000BC0243028F49F7049F4805E883020F041
:10227000C8010E947B0C9F2CF92C06C0D801159632
:102280009C91907F91F7F8CF8F2D61960FB6F894BF
:10229000DEBF0FBECDBFDF91CF911F910F91FF9099
:1022A000EF90DF90CF90BF90AF909F9008951F93D5
:1022B000CF93DF93CDB7DEB72C970FB6F894DEBF80
:1022C0000FBECDBF4F83588769877A878B879C87DE
:1022D000CE0107960E94870F8823D1F09F818885C1
:1022E0002A853B85232B31F08F3F31F481E09F3FDE
:1022F00019F403C081E001C080E080FD47C04F8138
:10230000588569857A858B859C850E94F90C3EC02D
:1023100086E0FE013796DE01119601900D928A95B6
:10232000E1F7FF81E8856A857B856115710531F0EC
:10233000EF3F31F481E0FF3F19F403C081E001C0B9
:1023400080E080FD23C02091E20130E0C9010196C8
:10235000877099274091E10150E084179507F1F1CA
:10236000F983EA837D836C8396E0929FD001939FEB
:10237000B00D1124AD51BE4FFE01319601900D926A
:102380009A95E1F78093E2010E94E00E16E08091B9
:10239000E1019091E201891771F1189FC0011124A8
:1023A0008D519E4F0E94870F882329F1E091E10112
:1023B0001E9FF0011124ED51FE4F40815181628139
:1023C0007381848195810E94F90C8091E10190E0F4
:1023D0000196877099278093E101D9CF0E94C30CA1
:1023E0001092E2011092E101E3E1F2E086E0DF0108
:1023F0001D928A95E9F72C960FB6F894DEBF0FBEB2
:10240000CDBFDF91CF911F910895809121028595D5
:102410008595859508958091210287700895909102
:102420002102977081E009F480E0089580912C02E8
:10243000089590912C02892B80932C020895809509
:1024400090912C02892380932C02089510922C02E3
:10245000089590912B02892B80932B0208958095EB
:1024600090912B02892380932B02089510922B02C6
:10247000089580912202089508950C943C120C94C2
:102480003D1290916E0292FD08C090912202981721
:1024900021F0809322020C943F1208958091220231
:1024A000882329F01092220280E00C943F120895B4
:1024B000CF93DF93E0910201F091030180912C0210
:1024C0008083E0910201F0910301908180912B02C1
:1024D000892B808380912202882381F0E091020180
:1024E000F09103019081892B80838091020190916A
:1024F00003010E94052681110E944E12C091020123
:10250000D091030148E050E069E172E0CE010E9401
:10251000522F892B69F088E0FE01A9E1B2E0019019
:102520000D928A95E1F7CE01DF91CF910C94902521
:10253000DF91CF9108950C943C1290916E0292FD20
:1025400010C098E0899F90011124262B209321022E
:102550000E947B0D809121028595859585950C942F
:102560009B120C947B0D1092210280E00C949B1224
:10257000209121028095822380932102982F9770C9
:1025800099F430E0482F082E000C550B241735071E
:1025900059F090916E0292FD07C0859585958595BD
:1025A0000E949C0D0C94B3120895CF9390916E02EB
:1025B00092FB222720F92817F9F0C82F892FC0FB9A
:1025C00082F980936E0280916D0290916E020E945A
:1025D000311382E00E94B81280913B0280FF0CC050
:1025E0001F92CF9385E291E09F938F930E945307B0
:1025F0000F900F900F900F90CF91089580916E02E1
:1026000082FB882780F991E089270C94D51281E01C
:102610000C94D51280E00C94D51280E090E00E94DA
:102620006D2F21E0893E9E4F09F020E0822F089512
:1026300082E090E00C945F2F83E090E00C945F2F99
:10264000CF9384E090E00E945F2FC82F82E290E059
:102650000E945F2F2C2F30E0A901582BCA01CF9187
:102660000895CF93C92F682F84E090E00E94732FC4
:102670006C2F82E290E0CF910C94732FAB01BC01E0
:1026800083E190E00C94852F60E070E0CB010C9426
:102690003E1369EE7EEF80E090E00E94912F60E0B3
:1026A00082E090E00E94732F60E083E090E00E945F
:1026B000732F1092DD011092DE011092DF01109253
:1026C000E00160E084E090E00E94732F60E082E22D
:1026D00090E00E94732F60E085E090E00E94732FED
:1026E00060E086E090E00E94732F6FEF87E090E05B
:1026F0000E94732F40E050E0BA0188E090E00E9411
:10270000852F60E08DE090E00E94732F40E050E064
:10271000BA0188E190E00E94852F60E087E190E0B7
:102720000E94732F40E050E0BA018CE190E00E94DB
:10273000852F60E070E080E290E00E94912F40E001
:1027400050E0BA0188E190E00E94852F0C945C076C
:102750000C944913682F8EE090E00C94732F0E9424
:10276000FB2660933702709338028093390290936E
:102770003A0260933302709334028093350290934F
:10278000360208950E94FB26609337027093380248
:102790008093390290933A0260932F027093300233
:1027A0008093310290933202089585B7806885BF87
:1027B00085B7806885BF089581E008950C94DC1387
:1027C00008950C94E0130C94E0130C94E3130C9410
:1027D000E0130C94E7130C94E0130E94D51382E0ED
:1027E00099E20E947A250E94EB130C94E9130E944F
:1027F000E1130C94E0130E9491160C9476080E9449
:10280000E6260E9468170E94FB130E94481E0E9441
:1028100027240C94E5138F929F92AF92BF92CF9290
:10282000DF92EF92FF920F931F93CF93DF93CDB779
:10283000DEB72A970FB6F894DEBF0FBECDBF0E9459
:102840007717982E81110E94AF138DE2A82E82E097
:10285000B82E00E010E0802E802F0E94B516D82EF2
:10286000F501C1905F01C826B1F40F5F1F4F023020
:10287000110589F78FEF89838A831B820E94EF26D7
:102880008160782F9D838C8349815A816B818D81F2
:102890000E94B9082FC080913B0281FD0E94BB16A7
:1028A000E12CFF24F3948C2D8F21F1F00E94DE1394
:1028B000882399F0EE828F82DF2081E009F480E0A6
:1028C00088870E94EF268160782F9A8789874E81BA
:1028D0005F8168858A850E94B908F801E35DFD4F34
:1028E0008081F826F08206C0E394FF0CF3E0EF123B
:1028F000DACFBBCF81E0911001C080E02A960FB6FD
:10290000F894DEBF0FBECDBFDF91CF911F910F9125
:10291000FF90EF90DF90CF90BF90AF909F908F90FF
:1029200008950E940B140E944E1F0E9439248111A9
:102930000E94C2130C948708CF93DF930E94B915AD
:10294000EC01811522E59207E8F5811531E5930741
:1029500008F0B6C0883E910528F5803E910508F044
:10296000E9C0883A910570F4853A910508F07AC07B
:102970008130910509F473C008F4D9C0049708F0B8
:10298000D9C0D5C08F3B910508F0D1C0C85AD0E05E
:10299000CC0FDD1FCB5ADE4F0990D881C02DCE0160
:1029A0009464C9C0811540E5940708F069C0811599
:1029B00050E4950708F060C09A9581159F4108F48E
:1029C000B9C0B5C0811536E5930728F5811545E5F1
:1029D000940708F092C0811554E5950708F087C068
:1029E000AC0143705527282F26952695C115D34550
:1029F00008F06CC081E090E002C0880F991F4A95F2
:102A0000E2F740E2249F90011124EC01C22BD32B6A
:102A1000CE019C6890C081152AE5920780F481154B
:102A200039E5930708F072C0811548E5940708F46A
:102A30007EC0D82FCC27CE01806F906A7CC0905684
:102A40008115904208F073C08D2F8F710E944D1632
:102A5000DD27D0628F71AE01582BCA016CC081E0B6
:102A600090E069C0C55AD0E0CD57DE4F8881C82FAD
:102A7000D0E0CE0190645FC0DF70CE01906A5BC091
:102A800074E0969587957A95E1F7282F23703C2F6F
:102A9000337081E090E002C0880F991F3A95E2F709
:102AA0009C68AC01522B9A019C2F9F70969596952D
:102AB00050E2959FE0011124C9018C2B9D2B3BC056
:102AC000D82FCC27CE01816F906A35C081E090E08D
:102AD00002C0880F991F4A95E2F750E2259F9001A6
:102AE0001124EC01C22BD32BCE019A6824C0D82F1D
:102AF000CC27CE01846F906A1EC00E944D168F7144
:102B000090E0D82FCC27CE01906215C08F700E9424
:102B10004D1694E0D695C7959A95E1F7CF70D0E021
:102B2000DC2FCC27D0699E01282BC90104C080E08E
:102B300090E001C0CE01DF91CF910895272F30E0C2
:102B4000F901EE0FFF1F2E0F3F1FF90196E0899F3D
:102B5000E00DF11D1124E60FF11DEE0FFF1FE852ED
:102B6000FF4F8591949108950E949E150E949C1498
:102B700008958238910569F1B0F48133910509F423
:102B80006DC048F48932910509F463C08A32910519
:102B900009F469C008958533910509F455C0893356
:102BA0009105B9F00895833E910569F138F4803EAE
:102BB0009105B1F0823E910509F10895863E910597
:102BC000A9F1873E9105B9F1843E910509F064C0F1
:102BD00023C020916D0220FD4FC021FD4DC00895FE
:102BE00080916D0280FD44C080916E0280FF44C0E0
:102BF00080916D0284FD42C083EE4DC080916D02D4
:102C000082FF38C0F5CF80916D0282FD33C0809184
:102C10006E0280FD31C0ECCF80916E0281FF32C028
:102C200080916D0284FD2AC087EE35C080916D02CF
:102C300083FF26C0F5CF80916D0283FD21C0809176
:102C40006E0281FD1FC0ECCF80916D0285FD1CC01E
:102C50001DC080916D0285FD19C016C080916D0266
:102C600086FD16C017C080916D0286FD13C010C08E
:102C700089E311C082EE0FC080EE0DC080E00BC072
:102C800086EE09C084EE07C089E205C085E303C073
:102C90008AE201C081E390E0089590916D0292FF75
:102CA0000DC0282F2871283019F4877F846006C052
:102CB000282F2471243011F48B7F886093FF0DC07E
:102CC000282F2871283119F4877E846106C0282FA7
:102CD0002471243111F48B7E886120916E0220FFD3
:102CE0000DC0382F3871383019F4877F816006C0E5
:102CF000382F3171313011F48E7F886021FF0DC083
:102D0000282F2871283119F4877E816106C0282F69
:102D10002171213111F48E7E886194FD877E0895A2
:102D200008950E940D13811102C00E94A8130E94F1
:102D3000181380933B020E94201390936E0280939D
:102D40006D020E9490160E941C13682F70E080E0B4
:102D500090E00E941B0D6091D9017091DA01809181
:102D6000DB019091DC010C94530DE82FF0E0EF585B
:102D7000FD4F80810895CF92DF92EF92FF920F93E3
:102D80001F93CF93DF9389E491E00E94BA0681E715
:102D9000E82E82E0F82EC0E0D0E094E4C92E91E065
:102DA000D92E0CE311E0DF93CF93DF92CF920E94F4
:102DB000530781E491E00E94BA06F70181917F01F7
:102DC0000E945D081F928F931F930F930E945307D9
:102DD0008AE391E00E94BA0621968DB79EB70896C5
:102DE0000FB6F8949EBF0FBE8DBFC230D105D9F685
:102DF000DF91CF911F910F91FF90EF90DF90CF90D7
:102E0000089508950C9401170C9402170C9401175F
:102E10000C940617CF93DF9346E851E0A1E0B0E0B1
:102E200020E030E0FA01E20FF31F80818F3FA1F034
:102E3000E82FE295EF70F0E061A18F70ED0102C024
:102E4000CC0FDD1F8A95E2F7CE019C2F909596233B
:102E500091A392A1892B82A32F5F3F4F233031058D
:102E600009F74D5F5F4FD1E04C385D07C9F6DF9140
:102E7000CF910895CF93DF93DC01462F50E083E09C
:102E8000689FF0011124EA57FE4F73E081E060E093
:102E900091919F3F99F0C92FC295CF70D0E028A1A2
:102EA00030E09F7002C0359527959A95E2F720FD96
:102EB00002C0282F02C020E030E0622B880F715042
:102EC00039F7FD01E40FF51F6083DF91CF9108957D
:102ED0000E940A17109272021092710210927002F0
:102EE00010926F0282E00E94AF170C94C5071F93E7
:102EF000CF93DF9300D0CDB7DEB71A82198260E09E
:102F0000CE0101960E943A1761E0CE0101960E941F
:102F10003A1742E050E0BE016F5F7F4F8FE692E0CC
:102F20000E94522F11E0009709F410E0892B31F034
:102F300089819A819093700280936F02212F42E0E1
:102F400061E772E08FE692E00E94B0170E94C70727
:102F5000812F0F900F90DF91CF911F9108950895C9
:102F6000FF920F931F93CF93DF938C01F62ED72FF1
:102F7000C42F222349F081E080933E020E94EF2675
:102F800090933D0280933C0280913E028823C1F0E1
:102F900080913C0290913D020E940727059780F0A6
:102FA000EF2DFD2FD8014C2F50E0CD01801B910B50
:102FB000841795071CF48D918193F7CF10923E02F0
:102FC000DF91CF911F910F91FF9008950E947E296C
:102FD0000E94FF130C948A290E948E290E9491144A
:102FE0000C94AC290E948D260E9465290E94ED1345
:102FF0000E94E6170E94EC170E94F713FBCFEF9296
:10300000FF920F931F93CF93DF938B01682F1111C2
:103010000AC0442329F0E82FF0E0E054FA4F64910D
:10302000762F862F75C0212F30E0E82FF0E0442363
:1030300021F0E054FA4FE491F0E046E0049FC00133
:103040001124CFEFD0E0BE010E94C42E4BEA46030C
:10305000C001479F900D1124800F911D800F911D7D
:10306000982F990F890FAE01421B530B4E9FD00131
:103070004F9FB00D5E9FB00D11249B2F189FA00194
:103080001124452F55278E01041B150B0E9FA001FF
:103090000F9F500D1E9F500D11247E01E81AF1085C
:1030A000E29E8001E39E100DF29E100D1124212F4F
:1030B0003327C21BD30BCE9F9001CF9F300DDE9FD5
:1030C000300D112462307105A9F048F461157105C5
:1030D00069F061307105C9F48B2F752F0DC0643014
:1030E000710581F058F06630710579F47E2F8B2FD1
:1030F000932F0DC0832F7B2F9E2F09C08E2F7B2FE8
:10310000952F05C08E2F732F02C07E2F852F692F1C
:10311000DF91CF911F910F91FF90EF90089541E0C3
:103120000E94FF17089508950E948F180895CF9365
:10313000DF93762FE901682F842F0E9494187983FA
:1031400068838A83DF91CF91089580917302282F3D
:10315000269530E02115310519F48170826005C093
:103160002532310524F081708864809373020895BC
:1031700088E090E00C94672FCF92DF92EF92FF925D
:103180006B017C010E94A518B701A60188E090E0C0
:10319000FF90EF90DF90CF900C94852FE3E7F2E063
:1031A00083E0808311828FEF828383831482608126
:1031B0007181828193810C94BC1880913B0280FFC5
:1031C00008C080E994E09F938F930E9453070F906B
:1031D0000F9080913B0280FF0FC08091730281703D
:1031E0001F928F9383E794E09F938F930E945307DE
:1031F0000F900F900F900F9080913B0280FF0FC0B7
:103200008091730286951F928F9388E594E09F9337
:103210008F930E9453070F900F900F900F90809103
:103220003B0280FF0EC0809174021F928F938EE349
:1032300094E09F938F930E9453070F900F900F90ED
:103240000F9080913B0280FF0EC0809175021F920B
:103250008F9384E294E09F938F930E9453070F9083
:103260000F900F900F9080913B0280FF0EC08091D5
:1032700076021F928F938AE094E09F938F930E942F
:1032800053070F900F900F900F9080913B0280FF9B
:103290000EC0809177021F928F938EEE93E09F93E2
:1032A0008F930E9453070F900F900F900F900895E7
:1032B0008091730280FF02C08695089580E0089592
:1032C00090917702933018F49F5F90937702882350
:1032D00051F0609173027091740280917502909127
:1032E00076020C94BC18089581E00C9460199091BA
:1032F0007702992319F0915090937702882351F027
:1033000060917302709174028091750290917602BF
:103310000C94BC18089581E00C94771970E00C941B
:10332000CB20609108018091730280FF0AC08091D8
:10333000070123E0829FC001112488589D4F0C94FF
:103340008E198091090190910A01891780F7E82F61
:10335000F0E09F01220F331FE20FF31FE858FD4FEB
:103360001182108212828F5FF0CF9091730290FFD2
:1033700016C09091090120910A01921770F4E92F6B
:10338000F0E0DF01AA0FBB1FEA0FFB1FE858FD4F5B
:103390008183608342839F5FF0CF0C9491190895DD
:1033A000CF93DF9300D01F92CDB7DEB79091730219
:1033B00090FF0AC09E012F5F3F4F0E9497184B81DC
:1033C00069818A810E94B5190F900F900F90DF914B
:1033D000CF910895CF93DF93EC01EC81F0E0E554B9
:1033E000FB4F4491E3E7F2E0628181810E94D019B2
:1033F0008C818F5F8C83DF91CF910895CF93DF9382
:10340000EC01E3E7F2E0438162818C810E94D019F4
:103410008C818F5F8C83DF91CF9108950F931F93E1
:10342000CF93DF9300D01F92CDB7DEB78C01809190
:103430003F0281110AC09E012F5F3F4F4FEF6FEF98
:103440000E9497188A8180933F02F801848181301D
:1034500051F028F0823061F440913F020AC080911F
:103460003F0240E007C060913F0240E080E003C0BF
:1034700040E080E060E00E94B519F801848190E0AE
:10348000019663E070E00E94D82E84830F900F9025
:103490000F90DF91CF911F910F9108954F925F92FE
:1034A0006F927F928F929F92AF92BF92CF92DF9254
:1034B000EF92FF920F931F93CF93DF9300D01F9251
:1034C000CDB7DEB7F82EB62EE42E622E90917302A1
:1034D00090FFB4C0E92FE695AE2FB0E0A457BE4FE1
:1034E0008C9180934B029E7F923061F49E012F5FFE
:1034F0003F4F8F2D0E9497184B8169818A810E94CE
:10350000B51962C0823019F4E09076025DC0863051
:1035100019F4F090740258C08930D9F3893109F058
:1035200053C0E9518E2F8170782E81E0A72CA826F8
:10353000E695F0E0E554FA4FC590D490412CDD2497
:1035400096ED892E91E0992E60910B014616D0F5EB
:10355000042D10E00C9DC0010D9D900D1C9D900D43
:10356000112470E00E94C42E5F2C711002C0560E10
:1035700001C0561A80913B0280FF11C0DF92CF92AA
:103580001F92AF921F925F921F924F929F928F92C3
:103590000E9453070FB6F894DEBF0FBECDBF8091D7
:1035A0000901080F111D9801220F331F020F131F6D
:1035B000980128583D4F4E2D6B2D852D0E94971850
:1035C0004394C2CF0E949119F0927402B092750296
:1035D000E09276026620E9F06091730270917402C5
:1035E00080917502909176020E94BC1880913B02F6
:1035F00080FF24C0809176021F928F938091750284
:103600001F928F93809174021F928F9381EB91E0B0
:103610000CC080913B0280FF11C01F92EF921F925D
:10362000BF921F92FF928AE891E09F938F930E942E
:1036300053070FB6F894DEBF0FBECDBF0F900F90AB
:103640000F90DF91CF911F910F91FF90EF90DF903E
:10365000CF90BF90AF909F908F907F906F905F9032
:103660004F900895E3E7F2E09181282F4381628132
:1036700088E0890F0C944E1A81E00C94321BE3E72A
:10368000F2E09181282F4381628188EF890F0C94A9
:103690004E1A81E00C943F1BE3E7F2E0628128E0E0
:1036A000620F08F46FEF282F438181810C944E1A2A
:1036B00081E00C944C1BE3E7F2E0628128E0621B9E
:1036C00008F460E0282F438181810C944E1A81E038
:1036D0000C945B1BE3E7F2E0438128E0420F08F41F
:1036E0004FEF282F628181810C944E1A81E00C9457
:1036F0006A1BE3E7F2E0438128E0421B08F440E064
:10370000282F628181810C944E1A81E00C94791BE0
:1037100021E00C944E1A20E00C944E1AFF920F9365
:103720001F93CF93DF93EC01F12C0FEF10E060912A
:103730000B01F616F0F4809109012F2D30E0280FCF
:10374000311DC901880F991F280F391F28583D4F77
:1037500070E0C8010E94D82E962F8C81409176028D
:1037600060917502F99E800D11240E949718F394C0
:10377000DECF0E9491199A818C8190FF02C08F5FE9
:1037800001C081508C83DF91CF911F910F91FF90E9
:103790000895BF92CF92DF92EF92FF920F931F9303
:1037A000CF93DF93FC01828180FF02C00FEF01C045
:1037B00001E010E080910B01181708F040C08091E3
:1037C0000901C12ED12CE601C80FD11DCE01880FF1
:1037D000991FC80FD91FC858DD4F198218821A8245
:1037E00034E0E32EF12CB12C809141028B0D853019
:1037F00014F0837005C087FF03C090910B01890FFF
:10380000082E000C990BC816D90691F48091760207
:103810008E9DA0018F9D500D11245595479555956E
:1038200047959E0160917502809174020E949718DD
:10383000B00EF1E0EF1AF108B9F61F5FBBCF0E949E
:10384000911980914102013031F4811102C08091BF
:103850000B01815007C090E0019660910B0170E070
:103860000E94D82E80934102DF91CF911F910F913A
:10387000FF90EF90DF90CF90BF900895CF9380910D
:10388000090190910A01891770F4E82FF0E09F0177
:10389000220F331FE20FF31FE858FD4F11821082F1
:1038A00012828F5FF0CFC0E060910B01C617C0F5A8
:1038B000EC2FF0E070E0CF010E94D82E209109019A
:1038C000820F20914002022E000C330B90E0E21791
:1038D000F307CCF020910601022E000C330B2E17BB
:1038E0003F078CF09C01220F331F820F931F9C0116
:1038F00028583D4F40917602609175028091740284
:103900000E9497180BC0FC01EE0FFF1F8E0F9F1F28
:10391000FC01E858FD4F118210821282CF5FC4CFA4
:103920000E9491192091050180914002820F80939D
:10393000400290910601920F9093060119165CF4D3
:10394000082E000C990B40910B0150E04150510999
:10395000841795071CF0219520930501CF910895B8
:103960008F929F92AF92BF92CF92DF92EF92FF928F
:103970000F931F93CF93DF938C01FC014481C42FDD
:10398000D0E09E01DE010E941C2F9B01AC010E9431
:10399000322F6B017C01E0E2F0E0EC1BFD0BA5E5B2
:1039A000B0E09B01AC010E94322F4B015C019F01F2
:1039B000DF010E94142F9B01AC010E943D2F9B014F
:1039C000AC012C0D3D1D4E1D5F1DC501B4010E94B3
:1039D000EC2EC22FD22F2A3228F4F3E02F9F900131
:1039E00011240DC025E530E02C1B3109C901880FD9
:1039F000991F280F391F37FF02C02F5F3F4F3595A2
:103A00002795C22FC095F12C85E5E82EED1A8091FF
:103A10000B01F816C8F4F1FC02C08E2D01C08D2FE9
:103A2000909109012F2D30E0290F311DA901440F7C
:103A3000551F240F351F28583D4F4C2F609175029C
:103A40000E949718F394E3CF0E949119F8018481A2
:103A5000811102C091E003C0803219F49FEF90936E
:103A6000040190910401890FF8018483DF91CF91C3
:103A70001F910F91FF90EF90DF90CF90BF90AF908C
:103A80009F908F9008950F931F93CF93DF93EC0136
:103A900000E010E080910B01282F30E0021713079F
:103AA00024F5909109019801290F311DA901440FB6
:103AB000551F240F351F28583D4F869590E04C81A7
:103AC000081719071CF4442331F002C0411103C048
:103AD0004091760201C040E06091750280917402CD
:103AE0000E9497180F5F1F4FD5CF0E9491198C81AC
:103AF00090E00196817099278C83DF91CF911F917F
:103B00000F91089560917302669570E04BE050E06C
:103B10008CE091E00E94452F892B19F481E080937D
:103B20004C020E94EF2690934302809342028091C0
:103B30003B0280FF08C081E791E09F938F930E9432
:103B400053070F900F90089510924C0280913B0202
:103B500080FF08C088E591E09F938F930E945307F0
:103B60000F900F9008959091730290FF54C0917040
:103B7000811102C0926006C0853210F0986402C0C4
:103B8000880F982B909373026623B1F060917302B3
:103B90007091740280917502909176020E94BC1817
:103BA00080913B0280FF1BC08091730286951F921B
:103BB0008F9384E393E00BC080913B0280FF0FC0A2
:103BC0008091730286951F928F9386E193E09F9375
:103BD0008F930E9453070F900F900F900F9060915A
:103BE0007302669570E04BE050E08CE091E00E943B
:103BF000452F892B19F00E94A41D02C00E94821D2E
:103C000081E0809345024091760260917502809137
:103C100074020C948B1B0895682F909173029695F3
:103C200081E0890F853208F081E00C94B31D81E0BA
:103C30000C940C1E682F9091730296958FEF890F4C
:103C400009F484E20C94B31D81E00C941A1E61E027
:103C50000C94B31D809173028160809373028091F4
:103C60003B0280FF0DC01F9281E08F9388EA92E0B3
:103C70009F938F930E9453070F900F900F900F9078
:103C80008091730286950C94271E60E00C94B31DFE
:103C900080914A02811160C080913B0280FF08C080
:103CA00087ED93E09F938F930E9453070F900F909F
:103CB00080913B0280FF08C081EC93E09F938F933B
:103CC0000E9453070F900F900E940D13811110C096
:103CD00080913B0280FF08C089E993E09F938F9316
:103CE0000E9453070F900F900E94A8130E94CE18B5
:103CF0000E94B818609373027093740280937502E7
:103D0000909376026E7FC1F480913B0280FF08C0E1
:103D100080E593E09F938F930E9453070F900F903D
:103D20000E94CE180E94B8186093730270937402B8
:103D300080937502909376020E94A5180E94DD1868
:103D400010924C028091730280FF03C086950E94FE
:103D5000451E81E080934A0208958091730281603C
:103D60008093730280913B0280FF0DC01F9281E01F
:103D70008F938FE692E09F938F930E9453070F904B
:103D80000F900F900F908091730286950C94451EB2
:103D9000109249028091480281110E94AD1E0C943C
:103DA000821D809173028E7F8093730260917302F3
:103DB0007091740280917502909176020E94BC18F5
:103DC00080913B0280FF0FC08091730281701F922F
:103DD0008F9387E392E09F938F930E9453070F90F6
:103DE0000F900F900F900E94A41D2FEF80E792E09C
:103DF000215080409040E1F700C000000C949119E0
:103E000080913B0280FF10C0809173028095817089
:103E10001F928F938FED92E09F938F930E94530791
:103E20000F900F900F900F908091730280FD0C9473
:103E3000D11E0C942A1E809173028E7F8093730290
:103E400080913B0280FF0CC01F921F928DEF91E08A
:103E50009F938F930E9453070F900F900F900F9096
:103E60000E94A41D2FEF80E792E0215080409040F7
:103E7000E1F700C000000C9491190E94A41D8091EC
:103E8000490281110AC081E0809349028091730246
:103E90008170809348020C941B1F08950F931F9309
:103EA000CF93DF9380914C02882309F485C08091E1
:103EB0004B02E0917302E695E81BE09344028230E6
:103EC00049F4F0E0E954FB4FE491CE2FD0E00AEE44
:103ED00019E149C0863049F4F0E0EC54FB4FE4911D
:103EE000CE2FD0E00EEF19E13EC0893051F4E695B7
:103EF000F0E0EF54FB4FE491CE2FD0E00EE81BE151
:103F000032C08F3051F4E695F0E0E255FB4FE4917A
:103F1000CE2FD0E009EC1BE126C0853149F4F0E05A
:103F2000E555FB4FE491CE2FD0E00EE31CE11BC022
:103F3000883181F0833239F4E9EAF4E0C591D49113
:103F40000EE01AE110C0843251F4C4EFD1E003E472
:103F50001DE109C0C8E2D0E000EB1CE104C0C0EDE7
:103F6000D7E003E918E180914502882361F01092BF
:103F700045020E94EF2690934302809342021092E2
:103F80004702109246020E94EF26E0914202F09111
:103F900043028E1B9F0B8F3F9F4770F4EC0FFD1F5A
:103FA000F0934302E093420282E492E0F801DF9151
:103FB000CF911F910F910994DF91CF911F910F9194
:103FC0000895882311F0FA0101C0FB010994CF93F1
:103FD000DF93C82FD62F0E9458198C1740F00E94EB
:103FE00058198D1720F4DF91CF910C94171E8C2F48
:103FF000DF91CF910C94271E1F93CF93DF93FB018A
:1040000012811111C3C0EC010E9416128272CD3CC4
:10401000FCE5DF0709F49AC0A8F5C73CECE5DE072C
:1040200009F476C0A8F4C43C9CE5D90709F45FC044
:1040300028F4C33CDC4509F457C054C0C53C9CE59A
:10404000D90709F459C0C63CDC4509F45CC04AC034
:10405000CA3CFCE5DF0709F46AC050F4C83CECE553
:10406000DE0709F45AC0C93CDC4509F45BC03AC01C
:10407000CB3C9CE5D90709F45FC0CC3CDC4509F496
:1040800060C030C0C23DFCE5DF0709F46FC088F4B2
:10409000CF3C9CE5D90709F460C008F45CC0C03D82
:1040A000FCE5DF0709F45CC0C13DDC4509F45BC0F9
:1040B00019C0C53D9CE5D90709F460C050F4C33D63
:1040C000FCE5DF0709F455C0C43DDC4509F454C0E4
:1040D00009C0C63D9CE5D90709F455C0CE35DD457C
:1040E00009F454C011E052C00E94001F4FC044E2C6
:1040F0005EE167E17EE104C047E15EE164E27EE10A
:104100000E94E11F43C049E45BE16CE37BE1F8CF2F
:104110004CE35BE169E47BE1F3CF47E65BE168E513
:104120007BE1EECF48E55BE167E67BE1E9CF45E87F
:104130005BE166E77BE1E4CF46E75BE165E87BE1D5
:10414000DFCF4BE859E164E779E1DACF44E759E1A1
:104150006BE879E1D5CF81E017C065E082E010C05F
:1041600068E086E00DC06EE089E00AC064E18FE09F
:1041700007C067E185E104C088E106C062E289E129
:104180000E94E71F03C083E20E94271E812FDF9158
:10419000CF911F910895539A2BB1277F3BB138607F
:1041A0004FB7F894FC01CB01880F991F680F791F56
:1041B0006E0F7F1FE617F70789F0819198E03BB9F2
:1041C000000000C087FF2BB9880F000000C000C0AE
:1041D00000C02BB900C09A9591F7ECCF4FBF8FE587
:1041E00094E00197F1F700C000000895CF93DF93AA
:1041F000EC01FB018281882309F43CC1C430FDE558
:10420000DF0760F4CB3F9CE5D90788F49E0122507C
:104210003C452431310508F02EC109C0C236EDE518
:10422000DE0729F0C63AFDE5DF0709F024C10E9448
:10423000201390936E0280936D02C1318CE5D807F4
:1042400009F4C6C008F042C0C930ECE5DE0709F445
:104250009BC000F5C5308CE5D80709F485C078F41B
:10426000C330ECE5DE0709F478C008F07AC0C2304C
:10427000DC4509F0F5C080916D028160EFC0C73068
:104280009CE5D90709F478C008F07AC080916D02E6
:104290008061E4C0CD30FCE5DF0709F487C058F445
:1042A000CB309CE5D90709F479C008F07BC0809138
:1042B0006D0288606FC0CF30FCE5DF0709F480C075
:1042C00008F082C080916D02877FC8C0CE3F9CE518
:1042D000D90709F471C000F5C531FCE5DF0709F421
:1042E00085C068F4C3319CE5D90709F475C008F0AE
:1042F00095C00E94C30C80916D028F77AFC0CC3FF8
:10430000FCE5DF07A9F108F054C0CB3FDC4509F01C
:10431000A7C080916E0240C0C230EDE5DE0709F40F
:1043200089C058F4C1158DE5D80709F45AC008F0C2
:1043300069C080916E0282602FC0C236EDE5DE0753
:1043400009F47CC0C63AFDE5DF0709F481C0C3303B
:10435000DD4509F085C080E06EC080916D0282600D
:104360007DC080916D0216C080916D02886076C01C
:1043700080916E0282604FC080916D0280626EC03B
:1043800080916D0280646AC00E94C30C80916D02AE
:10439000806864C0846062C081603DC080916D02AD
:1043A0008E7F5CC080916D028D7F58C080916D02C0
:1043B00016C080916E0218C080916E028D7F2BC056
:1043C00080916D028F7E4AC080916D028F7D46C0C4
:1043D00080916D028F7B42C080916D02877F8B7FC1
:1043E0003DC080916E028D7F8E7F15C080916D02E1
:1043F00082FB222720F991E0922790FB82F990FB23
:1044000083F92CC080916E02982F909591708E7FC9
:10441000892B90FB81F980936E0222C00E94C30C0D
:1044200080916D0287FB222720F991E0922790FB73
:1044300087F914C081E00E94AA1312C080916D0216
:1044400084FB222720F991E0922790FB84F906C093
:1044500080916D02982F909590FB80F980936D026A
:1044600080916D0290916E020E9431130E94C30CE4
:1044700080E001C081E0DF91CF910895CF93C82FF4
:104480001F928F9386EC96E09F938F930E94530721
:1044900081E090E0A0E0B0E0BC01CD0104C0660F77
:1044A000771F881F991FCA95D2F70E941B0D0F9086
:1044B0000F900F900F90CF910C94C30CEF92FF923E
:1044C0000F931F93CF93DF938B3109F4EDC008F066
:1044D0008EC08B3009F4B1C008F078C0863009F482
:1044E000AFC020F4853009F4BDC04EC1873009F457
:1044F000C0C0883009F048C10E941C131F928F93DE
:1045000084EE9AE09F938F930E9453070E941813A2
:1045100083FB992790F91F929F9382FB992790F92B
:104520001F929F9381FB992790F91F929F93982F39
:1045300091701F929F931F928F938BE99AE09F93A4
:104540008F930E9453070E94201387FB222720F994
:104550001F922F9386FB222720F91F922F9385FB12
:10456000222720F91F922F9384FB222720F91F92E4
:104570002F9383FB222720F91F922F9382FB222760
:1045800020F91F922F9391FB222720F91F922F933E
:10459000292F21701F922F9381FB222720F91F9230
:1045A0002F93282F21701F922F939F938F9386EB29
:1045B00099E09F938F930E9453078DB79EB788967B
:1045C0000FB6F8949EBF0FBE8DBF35C0803109F481
:1045D00095C020F48E3009F47BC0D6C0863109F432
:1045E000A8C0893109F0D0C086E397E084C08A3240
:1045F000E1F060F4873209F4C3C028F48E3108F486
:10460000C3C08D51BEC0893269F1BEC0833448F445
:104610008A3308F0B3C0853309F4B2C0883369F037
:10462000B3C0833409F4ACC0AFC08FE89BE00E94F4
:10463000BA060E94A813C1E0ACC083E198E05BC059
:1046400080913B02817F8E7F80933B0288EF97E0D1
:104650000E94BA068BE89BE00E94BA0681E0809334
:104660004D02E9CF8FE69BE00E94BA060E94CA077E
:10467000E2CF80913B02C82FC095C170C0FB80F98A
:1046800080933B02CC2329F083E69BE00E94BA068C
:1046900080C086E59BE00E94BA0680913B02897F3C
:1046A000877F80933B02C7CF90913B0291FBCC2741
:1046B000C0F981E0C827892FC0FB81F980933B02B4
:1046C000CC2319F089E49BE029C08BE39BE013C065
:1046D00090913B0292FBCC27C0F981E0C827892F3B
:1046E000C0FB82F980933B02CC2319F08CE29BE063
:1046F00015C08CE19BE00E94BA069DCF90913B02D1
:1047000093FBCC27C0F981E0C827892FC0FB83F930
:1047100080933B02CC2351F080E19BE00E94BA06DB
:1047200080913B02816080933B0233C083E09BE039
:10473000E2CF0E94FB26162F072FF82EE92ED091EC
:104740006C02C09123010E948425EF92FF920F9387
:104750001F931F92DF931F92CF931F928F938BEC27
:1047600096E09F938F930E9453078DB79EB70C9648
:104770000FB6F8949EBF0FBE8DBF5DCF895301C0A9
:1047800080E00E943E2257CF81E09BE00E94BA0663
:10479000C0E08C2FDF91CF911F910F91FF90EF9090
:1047A000089580E008950C94D123CF93C82F809171
:1047B0004D02882319F0813031F038C00E94161262
:1047C0008232B1F504C00E941612823261F48C2F3D
:1047D0000E94D323811104C08C2F0E945E2224C02A
:1047E00081E090E021C08C2F0E94D12381111BC059
:1047F000C43189F018F4CB3029F010C0C93259F017
:10480000C83361F488EF97E00E94BA0682EC96E024
:104810000E94BA0608C010924D020CC080EC96E0CF
:104820000E94BA0607C081E0817006C010924D0256
:1048300080E002C080E0F8CFCF9108958FE891E04A
:104840000197F1F700C0000008950C946807519893
:10485000599A5098589A0E941E2489B18695817061
:10486000489902C090E001C092E0892B80935002E9
:104870000895E0915002EE0FEE0FE093500229B13F
:1048800021FB882780F990E0489903C020E030E0C0
:1048900002C022E030E0822B932B8E2B80935002BB
:1048A0008F70E82FF0E0EF54FE4F908180914F021F
:1048B000890F80934F0284305CF080914E028F5FAD
:1048C00080934E0260E080E00E94252421E001C038
:1048D00020E080914F028D3F54F480914E02815030
:1048E00080934E0261E080E00E94252421E08091C7
:1048F0004F02082E000C990B64E070E00E94D82E45
:1049000080934F02822F0895CF93DF9386319C4589
:1049100041F5EB010E941612982F8A812091020125
:1049200030910301882379F09A7A81E009F480E0DC
:1049300080935102911102C069E201C065E3C9018F
:104940000E9447260AC080915102811102C069E28B
:1049500001C065E3C9010E9449260E94581280E007
:1049600001C081E0DF91CF9108950F931F93CF9302
:10497000DF93C42FD22FFC0182818823C9F040939A
:1049800054020E94EF26909353028093520280E2D9
:104990008C0F883008F057C0C77081E001C0880FC5
:1049A000CA95EAF7DF91CF911F910F910C942F0ACE
:1049B00080915402481330C080915202909153026A
:1049C0000E940727883C910538F510E21D0FCD178E
:1049D000B9F080E28C0F883040F4C77081E001C0EC
:1049E000880FCA95EAF70E94360A183028F581E048
:1049F0009D2F977001C0880F9A95EAF70E942F0AA1
:104A0000802F0E94260A1830F0F4D77081E001C090
:104A1000880FDA95EAF70AC080E28C0F883098F4A4
:104A2000C77081E001C0880FCA95EAF7DF91CF9186
:104A30001F910F910C94360A802FDF91CF911F9117
:104A40000F910C94260ADF91CF911F910F91089539
:104A50000F939C01CB01243F4CE5340731F188F4DE
:104A6000293DFCE53F07D9F02A3D4CE5340779F1B3
:104A7000283D3C45A9F506E221EE41EE68ED7CE5D6
:104A80002BC0263FFCE53F07E1F0A8F0273F3C455F
:104A900039F507E225EE46EE67EF7CE51DC007E23B
:104AA00025EE45EE69ED7CE517C006E221EE40EE0D
:104AB00064EF7CE511C007E225EE44EE65EF7CE58E
:104AC0000BC006E221EE42EE66EF7CE505C008E28F
:104AD00021E045EE6AED7CE50E94B52480E008C047
:104AE000FC018281882319F01092540201C081E0F8
:104AF0000F9108959093D1018093D00108959093E0
:104B00005A02809359020895E0915902F0915A0295
:104B1000309721F00190F081E02D099480E0089514
:104B2000EF92FF920F931F93CF93DF93E09159027F
:104B3000F0915A023097B1F18C010280F381E02D9F
:104B4000099580913B0282FF2DC080FF04C088EA56
:104B50009BE00E94BA06E80118E082EAE82E8BE0AA
:104B6000F82E80913B0280FF0BC088811F928F93AB
:104B7000FF92EF920E9453070F900F900F900F90AB
:104B8000115021961111EDCF80913B0280FF0AC098
:104B900080EA9BE0DF91CF911F910F91FF90EF9002
:104BA0000C94BA06DF91CF911F910F91FF90EF9077
:104BB000089520915702309158022817390771F053
:104BC0009093580280935702E0915902F0915A0253
:104BD000309721F00680F781E02D09940895209107
:104BE0005502309156022817390771F090935602FA
:104BF00080935502E0915902F0915A02309721F0CA
:104C00000084F185E02D09940895FC01329697E027
:104C100080E0915029F021912223D9F38F5FF9CFC1
:104C20000895662349F0FC01329608962191621797
:104C300029F0E817F907D1F780E0089581E0089599
:104C40009C01FC0132969FEF80E04191461789F06C
:104C50009F3F19F4411101C0982F8F5F8630A9F74B
:104C60009F3F39F0F901E90FF11D97FDFA95628335
:104C7000089508959C012A5F3F4FFC01428146132D
:104C800001C01282019682179307B9F708950C9418
:104C900020260C943A26029626E0FC0111922A95D1
:104CA000E9F7089508950C94522683E080935B02FF
:104CB0000C945326811102C081E001C082E08093F0
:104CC0005B020C9453260C945A2681E080935B027D
:104CD0000C9453260C94652608950C946C260C9421
:104CE0006D260C946C260C946C260C946C260E94F9
:104CF00073260E9477170E94712680E00E94B516E5
:104D0000811108C081E00E94B51691E0811103C0B5
:104D100090E001C091E0892F089508951F920F92AD
:104D20000FB60F9211248F939F93AF93BF938091EF
:104D30005C02811113C08091840290918502A09140
:104D40008602B09187024196A11DB11D8093840215
:104D500090938502A0938602B0938702BF91AF9192
:104D60009F918F910F900FBE0F901F90189580917B
:104D70008C02843031F10E94510810925C0220E4D0
:104D800088E190E00FB6F894A895809360000FBE7C
:104D90002093600083B7817F846083BF83B7816085
:104DA00083BF7894889583B78E7F83BF0FB6F894BE
:104DB000A8958091600088618093600010926000E7
:104DC0000FBE08950E94C30C0C94570882E084BD66
:104DD00093E095BD9AEF97BD80936E0008952FB72D
:104DE000F8948091840290918502A0918602B091FE
:104DF00087022FBF08952FB7F894609184027091B5
:104E0000850280918602909187022FBF08959C01B0
:104E10004FB7F8948091840290918502A091860208
:104E2000B09187024FBF821B930B089578941F9215
:104E30000F920FB60F9211248F939F93AF93BF934E
:104E40008091840290918502A0918602B0918702A0
:104E50000196A11DB11D8093840290938502A093B9
:104E60008602B0938702BF91AF919F918F910F906F
:104E70000FBE0F901F90189587E797E79093010852
:104E8000809300089AE088E10FB6F894A895809383
:104E900060000FBE90936000FFCF80916B02089579
:104EA0000895CF93DF9321E02093E9002FEF309115
:104EB000E800215035FD06C035ED3A95F1F70000C8
:104EC0002111F5CF2091E80025FF14C0EC0140E04E
:104ED00050E068E070E00E941B2A8091E8008E7725
:104EE0008093E80088E0FE01A3E6B2E001900D9215
:104EF0008A95E1F7DF91CF91089580935F027093D7
:104F000061026093600280918C02843001F582E03E
:104F10008093E9008FEF9091E800815095FD06C0E5
:104F200095ED9A95F1F700008111F5CF8091E80099
:104F300085FF0DC040E050E063E070E08FE592E057
:104F40000E941B2A8091E8008E778093E8000895E4
:104F5000BC0184E00C947D27BC0183E00C947D2788
:104F600008958EEC9BE00E94BA0680918B0281111D
:104F700009C00E94AC2B0E94092C8091E200846041
:104F80008093E20008958AEC9BE00E94BA0610929A
:104F90008B02089586EC9BE00E94BA060C946A2668
:104FA00082EC9BE00E94BA066091880281E0611168
:104FB00001C080E00C9455268EEB9BE00E94BA065F
:104FC00090918C0281E0943009F080E06091880239
:104FD0000C945A2620915E022F5F822F62E30E947A
:104FE000B82E992319F020935E02089510925E0264
:104FF00080916202882371F180918C02843041F5A6
:105000008091E9008F702091EC00922F917020FD2B
:1050100090E8892B93E09093E9009091EB0090FF4A
:1050200014C09091EE0097FF10C09091E80095FF9A
:1050300003C01092F100F9CF9091E80090FF05C0F5
:105040009091E8009E779093E8008F708093E9003C
:1050500010926202089542E061EC81E00E94252BEB
:1050600042E261EC82E00E94252B42E261EC83E0A7
:105070000E94252B90918C0281E0943009F080E011
:10508000609188020C94632680918E02833009F42B
:1050900061C030F4813071F0823009F49AC0089513
:1050A0008A3009F486C08B3009F46CC0893009F06D
:1050B000A8C020C080918D02813A09F0A2C08091E1
:1050C000E800877F8093E80080919102909192029E
:1050D000892B21F468E083E692E003C060E080E081
:1050E00090E070E00E94662A8091E8008B778093C0
:1050F000E800089580918D02813209F082C080918C
:10510000910290919202029708F07BC08091E80092
:10511000877F8093E8008091E80082FD05C0809140
:105120008C028111F8CF6DC02091F3008091F200C4
:1051300090E0922B029731F48091F100813011F0D0
:10514000863021F48091F10080936B028091E80019
:105150008B7753C080918D02813A09F052C08091C3
:10516000910290919202892B09F04BC08091E80046
:10517000877F8093E8008091E80080FFFCCF8091DA
:10518000230136C080918D028132D9F58091910240
:1051900090919202892BA9F58091E800877F8093F6
:1051A000E8000E945A2B80918F02809323010C9477
:1051B000C30C80918D02813221F58091E800877FB8
:1051C0008093E8000E945A2B8091900280936C0299
:1051D000089580918D02813AA1F48091E800877F43
:1051E0008093E8008091E80080FFFCCF80916C0202
:1051F0008093F1008091E8008E778093E8000C9412
:105200005A2B08959FB7F894109262029FBF909115
:105210008C02943009F057C09091E9009F70309152
:10522000EC00232F217030FD20E8922B23E0209307
:10523000E9002091EB0020FF43C02091EE0027FF02
:105240003FC020915D02222321F02091E80025FF3C
:1052500037C010925D0226E03091E80035FD15C0A0
:1052600030918C02343061F53091EB0035FD28C06F
:10527000215021F481E080935D0222C0EFE9FFE03C
:105280003197F1F700C00000E7CF8093F1008091E3
:10529000E80085FD0AC08091E80080FFFCCF809186
:1052A000E8008E778093E80006C08FB7F89421E07D
:1052B000209362028FBF9F709093E90080E0089571
:1052C0009F709093E9008FEF089584B7877F84BF24
:1052D0000FB6F894A8958091600088618093600073
:1052E000109260000FBE90E080E80FB6F8948093B3
:1052F0006100909361000FBE0C9465260E94AC2B58
:105300000E94092CE2EEF0E0808184608083789432
:105310000C949D2E87E191E00C947F2580918C0266
:105320008530C9F48AEB9BE00E94BA0680918C021A
:10533000853079F40E94B72680918A028823B1F3E0
:105340000E947726882391F30E94052A0E94C30CAD
:10535000EDCF0C94E226089508950C94AF29292FDF
:10536000332723303105C9F060F42130310581F055
:105370002230310509F041C08BE590E02CE13CE0A2
:1053800040C021323105E1F02232310531F135C022
:1053900082E190E027E73CE034C099278130910515
:1053A00049F028F0029749F5E2EDFBE005C0E8E19D
:1053B000FCE002C0E0E0FCE0849190E09F0121C0AD
:1053C00063307105D0F4660F771FFB01E653FE4F83
:1053D0002081318189E090E014C06330710568F468
:1053E000FB01EE0FFF1FEC53FE4F20813181FB01CB
:1053F000EF53FE4F808190E004C080E090E020E019
:1054000030E0FA0131832083089580E189BD82E193
:1054100089BD09B400FEFDCF8091D8008F7D8093B7
:10542000D8008091E00082608093E0008091E000ED
:1054300081FDFCCF0895CF92DF92EF92FF920F9300
:105440001F93CF93DF93EC018B017A010E94792B9C
:10545000811133C0E114F10439F0F70180819181A9
:10546000081B190BC80FD91FC12CD12C0115110510
:1054700019F18091E80085FD16C08091E8008E77D3
:105480008093E800E114F10449F0F70180819181F3
:10549000C80ED91ED182C08285E00FC00E94792B30
:1054A000882321F30AC089918093F10001501109EA
:1054B000FFEFCF1ADF0ADACF80E0DF91CF911F91A3
:1054C0000F91FF90EF90DF90CF900895209193027D
:1054D000309194022617370748F06115710539F4A9
:1054E0002091E8002E772093E80001C0B901FC016B
:1054F00020E06115710579F180918C028823F1F12A
:105500008530F1F18091E80083FD3CC08091E80096
:1055100082FD2EC08091E80080FFEBCF2091F30048
:105520008091F20090E0922B6115710551F0883066
:10553000910538F421912093F10061507109019691
:10554000F3CF21E0089709F020E08091E8008E7702
:105550008093E800CECF2111CFCF0AC080918C027A
:10556000882361F0853061F08091E80083FD0AC0F6
:105570008091E80082FFF2CF80E0089582E00895F4
:1055800083E0089581E00895209193023091940280
:105590002617370748F06115710539F42091E800A6
:1055A0002E772093E80001C0B901FC0120E06115CD
:1055B000710591F180918C02882309F440C08530F7
:1055C00009F43FC08091E80083FD3DC08091E80070
:1055D00082FD2FC08091E80080FFE9CF2091F30089
:1055E0008091F20090E0922B6115710559F088309E
:1055F000910540F424912093F10031966150710996
:105600000196F2CF21E0089709F020E08091E800B0
:105610008E778093E800CBCF2111CCCF0AC0809148
:105620008C02882361F0853061F08091E80083FD71
:105630000AC08091E80082FFF2CF80E0089582E006
:10564000089583E0089581E00895982F973068F5D4
:105650009093E900981739F07091EC002091ED00DB
:105660005091F00003C0242F762F50E021FD02C09E
:105670009F5FECCF3091EB003E7F3093EB00309199
:10568000ED003D7F3093ED003091EB0031603093C1
:10569000EB007093EC002093ED005093F00020910C
:1056A000EE0027FDE5CF80E008958F708093E9003C
:1056B00081E0089580918D0287FF11C08091E800FC
:1056C00082FD05C080918C028111F8CF11C08091BC
:1056D000E8008B770BC080918C02882349F0809181
:1056E000E80080FFF8CF8091E8008E778093E80093
:1056F00008952091E4003091E50095E64091EC009A
:10570000842F817040FF23C08091E80080FD1DC080
:1057100080918C02882399F0853099F08091EB007C
:1057200085FD11C04091E4005091E5002417350734
:1057300029F3915011F09A01E1CF84E0089582E0BD
:10574000089583E0089581E0089580E008954091F0
:10575000E80042FFDDCF08950E941A2C0E94222CFF
:10576000E0EEF0E0808181608083E8EDF0E0808110
:105770008F77808319BCA7EDB0E08C918E7F8C93DE
:1057800080818F7E808310928B0208950F931F93E8
:10579000CF93DF930E941A2C0E94222CC8EDD0E0F8
:1057A00088818F77888388818068888388818F7DCE
:1057B000888319BC10928C021092880210928A027F
:1057C0001092890200EE10E0F80180818B7F8083C7
:1057D00088818160888342E060E080E00E94252B20
:1057E000E1EEF0E080818E7F8083E2EEF0E0808168
:1057F00081608083808188608083F80180818E7FD2
:105800008083888180618883DF91CF911F910F9180
:105810000895E8EDF0E080818F7E8083E7EDF0E091
:1058200080818160808384E082BF81E080938B02ED
:105830000C94C62BE8EDF0E080818E7F808310927F
:10584000E20008951092DA001092E10008951F928C
:105850000F920FB60F9211242F933F934F935F93A4
:105860006F937F938F939F93AF93BF93EF93FF9328
:105870008091E10082FF0BC08091E20082FF07C0AF
:105880008091E1008B7F8093E1000E94EA27809164
:10589000DA0080FF1FC08091D80080FF1BC080917C
:1058A000DA008E7F8093DA008091D90080FF0DC0EE
:1058B00080E189BD82E189BD09B400FEFDCF81E0B0
:1058C00080938C020E94B12705C019BC10928C02F3
:1058D0000E94C3278091E10080FF19C08091E200FF
:1058E00080FF15C08091E2008E7F8093E20080915E
:1058F000E20080618093E2008091D8008062809312
:10590000D80019BC85E080938C020E94D02780913A
:10591000E10084FF30C08091E20084FF2CC080E170
:1059200089BD82E189BD09B400FEFDCF8091D80018
:105930008F7D8093D8008091E1008F7E8093E1007D
:105940008091E2008F7E8093E2008091E20081608E
:105950008093E20080918802882311F084E007C0E0
:105960008091E30087FD02C081E001C083E0809365
:105970008C020E94DC278091E10083FF29C0809186
:10598000E20083FF25C08091E100877F8093E100E2
:1059900082E080938C02109288028091E1008E7FD9
:1059A0008093E1008091E2008E7F8093E2008091FD
:1059B000E20080618093E20042E060E080E00E94CB
:1059C000252B8091F00088608093F0000E94CA2708
:1059D000FF91EF91BF91AF919F918F917F916F91C7
:1059E0005F914F913F912F910F900FBE0F901F909D
:1059F00018951F920F920FB60F9211242F933F9379
:105A00004F935F936F937F938F939F93AF93BF93C6
:105A1000CF93DF93EF93FF93C091E900CF70809114
:105A2000EC00D82FD17080FDD0E81092E900809171
:105A3000F000877F8093F00078940E943D2D1092B3
:105A4000E9008091F00088608093F000CD2BCF704A
:105A5000C093E900FF91EF91DF91CF91BF91AF919A
:105A60009F918F917F916F915F914F913F912F9176
:105A70000F900FBE0F901F9018951F93CF93DF9339
:105A8000CDB7DEB7AA970FB6F894DEBF0FBECDBF75
:105A9000EDE8F2E08091F100819322E0E539F20730
:105AA000C9F70E9444288091E80083FF2EC18091AD
:105AB0008D0290918E02492F50E04A30510508F036
:105AC00024C1FA01EE59FF4F0C940E2F803821F0BB
:105AD000823809F01AC108C08091890290918A0227
:105AE000992389F082600FC0809191028F70873076
:105AF00008F00BC18093E9008091EB0085FB8827BB
:105B000080F91092E9009091E800977F9093E80067
:105B10008093F1001092F100D1C0282F2D7F09F061
:105B2000F4C0882319F0823061F0EFC080918F02B9
:105B3000813009F0EAC0933009F080E080938A0256
:105B40002EC080918F0281112AC0809191028F70A6
:105B50002FEF280F263008F0D8C08093E90020915D
:105B6000EB0020FF1CC0933021F48091EB00806299
:105B700014C09091EB0090619093EB0021E030E035
:105B8000A90102C0440F551F8A95E2F74093EA002D
:105B90001092EA008091EB0088608093EB001092F5
:105BA000E9008091E800877F8093E8000E945A2BEB
:105BB000ACC08111AAC010918F021F778091E300C1
:105BC0008078812B8093E3008091E800877F809329
:105BD000E8000E945A2B8091E80080FFFCCF809162
:105BE000E30080688093E300111102C082E001C0ED
:105BF00083E080938C0289C08058823008F085C091
:105C000080918F02909190028C3D53E0950779F539
:105C100083E08A838AE289834FB7F894DE01139682
:105C200020E03EE051E2E32FF0E050935700E49192
:105C300020FF03C0E295EF703F5FEF708E2F90E082
:105C4000EA3010F0C79601C0C0968D939D932F5FE8
:105C5000243149F74FBF8091E800877F8093E800A7
:105C60006AE270E0CE0101960E94662A16C0609139
:105C7000910270919202AE014F5F5F4F0E94AD2979
:105C8000BC01892B09F441C09091E800977F909363
:105C9000E80089819A810E94C42A8091E8008B776C
:105CA0008093E80032C0803881F58091E800877FDA
:105CB0008093E800809188028093F1008091E80051
:105CC0008E7772CF811121C080918F0290919002C6
:105CD00099270297D4F48091E800877F8093E800A9
:105CE00080918F02809388020E945A2B80918802B3
:105CF000811106C08091E30087FD02C081E001C0F0
:105D000084E080938C020E942B288091E80083FF1E
:105D10000AC08091E800877F8093E8008091EB00C3
:105D200080628093EB00AA960FB6F894DEBF0FBE98
:105D3000CDBFDF91CF911F910895CF9380918C02B9
:105D40008823A1F0C091E900CF709091EC00892FD9
:105D5000817090FD80E8C82B1092E9008091E800E6
:105D600083FD0E943D2DCF70C093E900CF9108952F
:105D7000991B79E004C0991F961708F0961B881F9D
:105D80007A95C9F780950895AA1BBB1B51E107C0FE
:105D9000AA1FBB1FA617B70710F0A61BB70B881FBB
:105DA000991F5A95A9F780959095BC01CD0108954A
:105DB00097FB072E16F4009407D077FD09D00E94B8
:105DC000C42E07FC05D03EF4909581959F4F089511
:105DD000709561957F4F0895A1E21A2EAA1BBB1BF7
:105DE000FD010DC0AA1FBB1FEE1FFF1FA217B307A7
:105DF000E407F50720F0A21BB30BE40BF50B661FBD
:105E0000771F881F991F1A9469F760957095809580
:105E100090959B01AC01BD01CF010895EE0FFF1FCE
:105E20000590F491E02D09940E941C2F332312F465
:105E30008A1B9B0B0C942D2FA29FB001B39FC00116
:105E4000A39F700D811D1124911DB29F700D811DA6
:105E50001124911D08950E941C2FB7FF0895821BE5
:105E6000930B08950E941C2FA59F900DB49F900D39
:105E7000A49F800D911D11240895B7FF0C94322F1B
:105E80000E94322F821B930B0895FC014150504019
:105E900030F001900616D1F73197CF010895882789
:105EA00099270895FB01DC0104C08D9101908019B0
:105EB00021F441505040C8F7881B990B0895F99977
:105EC000FECF92BD81BDF89A992780B50895A6E1CD
:105ED000B0E044E050E00C94992FA8E1B0E042E03B
:105EE00050E00C94992F262FF999FECF92BD81BDD9
:105EF000F89A019700B4021639F01FBA20BD0FB608
:105F0000F894FA9AF99A0FBE08950396272F0E94E3
:105F1000742F0E94732F252F0E94742F242F0C940E
:105F2000742F0196272F0E94742F0C94732FDC017D
:105F3000CB01FC01F999FECF06C0F2BDE1BDF89A94
:105F4000319600B40D9241505040B8F70895F8943E
:025F5000FFCF81
:105F5200C8002302010102000400040401191A1BF3
:105F62001C1D1E1F2021224D275127B027AC27A818
:105F720027502701E200E900EA00B500B600B700A9
:105F8200CD008301CC008A019201940121022302F7
:105F920024022502260227022A02B300B4006F005F
:105FA2007000818283E200E900EA00B500B600B722
:105FB20000CD008301CC008A0192019401210223C9
:105FC2000224022502260227022A02B300B4006F2D
:105FD200007000818283973192C63432000102023E
:105FE20002020606060909090909090F0F0F0F0F18
:105FF2000F1515151819191919191919191919231C
:106002002400FF0100010000FFFF0000010001FF6A
:1060120000403222DD0CAB0C890C2E0C470C600CBC
:00000001FF
